:100000000C9420030C9464030C9464030C94640318
:100010000C9464030C9464030C9464030C946403C4
:100020000C9464030C9464030C94FE0D0C94D00E99
:100030000C9464030C9464030C9464030C946403A4
:100040000C9464030C94DA220C9464030C946403FF
:100050000C9464030C946D1C0C9464030C94640362
:100060000C9464030C9464030C9464030C94640374
:100070000C9464030C9464030C9464030C94640364
:100080000C9464030C9464030C9464030C94640354
:100090000C9464030C9464030C9464030C94640344
:1000A0000C9464030C9464030C9464033D0F5F0F81
:1000B0004D105F0F4D10A40FC70F4D101C102F10C7
:1000C000FE12FE122D132D1363138313B414B414F4
:1000D0008E13B4143E143E14A514B414B414AE1408
:1000E0004B144B144B144B144B144B144B144B1418
:1000F0004B144B144B144B144B144B144B144B1408
:100100005D146A1471147814821429002B000354AE
:10011000E100354100001E000E000B001B71640061
:100120004D001F00370004001400E1044C002000C3
:1001300012000800340050002A00210036000C0094
:100140002F004F004A0022001D001800330000005D
:100150000254E000E3000000E20000002E77E4001B
:10016000E7000000E60000002E7F230019000700D2
:1001700005000000045424000A0017001300520078
:100180004B002500060015001A0051002C00260027
:100190000F0011001000E108280027002D001600B4
:1001A0000D7130004E0038001C000942E50031415D
:1001B00000000100010001000100010000003A0000
:1001C000350031000100010001003B003502210231
:1001D000640001004C003C001E02240622020100C3
:1001E00001003D002D0224022404010001003E0014
:1001F00001003700110400000100010001000000AF
:1002000001000000010001000100000001000000E9
:1002100001003F00240624022302000001004000E8
:1002200022042502350001000100410023042602BA
:100230003502370001004200240425041F021E027B
:100240000100430031002604310201000100440096
:10025000450001002D020100000001000100010025
:10026000010001000000010001000100FB0001008D
:10027000010001000100F200F9000100010001008D
:10028000F000F100FA00F400010001000100F300A9
:10029000FC00F5000100010001000100F600000073
:1002A0000100010001000000010000000100010048
:1002B0000100000001000000010001000100010038
:1002C000010000000100010001000100A800A900D8
:1002D0000100010001000100AC00AA00B60001000D
:1002E00001000100AB00500001000100010001000D
:1002F000520051000100AE000100010001004F005A
:10030000000029002B000100E100354100001E0023
:10031000140004001D7164004D001F001A00160037
:100320001B00E1044C0020000800070006005000FC
:100330002A0021001500090019004F004A00220080
:1003400017000A000500000001001908E300000082
:10035000E20000002E770608E7000000E60000003B
:100360002E7F23001C000B00110000000100240060
:1003700018000D00100052004B0025000C000E006C
:10038000360051002C00260012000F003700E10853
:100390002800270013003300387130004E002D0074
:1003A0002F003442E500314100000100010001004E
:1003B0000100010000000100010001000100010036
:1003C00001000100010050000100010001000100D6
:1003D00052005100010001000100010001004F0026
:1003E0000100010001000100010001000100000006
:1003F00001000100010000000100000001000100F7
:10040000010000000100000001003F005200510007
:100410002302000001004000240021001E002700EC
:1004200001004100250022001F00370001004200AA
:100430002600230020002700010043003002300086
:1004400024022E00010044004500010001000100CB
:10045000000016034500720067006F0044006F0043
:100460007800200045005A00000016034500720085
:1004700067006F0044006F007800200045005A00BC
:1004800000000403090409026D00040100A0FA0938
:100490000400000103010100092111010001223FB4
:1004A000000705810308000A090401000103010295
:1004B00000092111010001224D00070582030800F7
:1004C0000A090402000103000000092111010001D2
:1004D0002236000705830308000A0904030001030C
:1004E00000000009211101000122390007058403E1
:1004F0001000011201100100000008EDFE071301B9
:10050000000102000105010906A101050719E02902
:10051000E7150025019508750181020508190129D3
:10052000059505750191029501750391010507195E
:1005300000297715002501957875018102C0050114
:100540000980A101850216010026B7001A01002AC0
:10055000B700751095018100C0050C0901A1018546
:1005600003160100269C021A01002A9C02751095B0
:10057000018100C005010902A1010901A1000509CD
:1005800019012905150025019505750181029501BF
:10059000750381010501093009311581257F950217
:1005A0007508810609381581257F95017508810632
:1005B000050C0A38021581257F950175088106C052
:1005C000C005010906A101050719E029E715002565
:1005D00001950875018102950175088101050819C9
:1005E0000129059505750191029501750391010594
:1005F00007190029FF150025FF950675088100C021
:100600000000000000000000000000010204060AD3
:100610000F17202C3A4A5D71879DB3C7DAE9F5FCC4
:10062000FFFCF5E9DAC7B39D87715D4A3A2C2017C4
:100630000F0A060402010000000000000000000094
:1006400011241FBECFEFDAE0DEBFCDBF04B603FE3C
:1006500024C08091FB019091FC01A091FD01B0911B
:10066000FE018730904BA740B04BB9F41092FB01CC
:100670001092FC011092FD011092FE0114BE84B78D
:10068000877F84BF88E10FB6F89480936000109252
:1006900060000FBEE0E0FFE3099511E0A0E0B1E0EB
:1006A000E2E4F9E402C005900D92A433B107D9F752
:1006B00011E0A4E3B1E001C01D92AB3FB107E1F747
:1006C0000E94420B0C949F240C9400001092B900DD
:1006D0008AE08093B800089594EA9093BC009091CA
:1006E000BC0097FFFCCF9091B900987F983021F023
:1006F000903111F081E008958093BB0084E88093ED
:10070000BC008091BC0087FFFCCF8091B900887F3E
:10071000883111F0803471F780E0089584E9809386
:10072000BC008091BC0084FDFCCF08958093BB0089
:1007300084E88093BC008091BC0087FFFCCF90913F
:10074000B900987F81E0983209F480E0089584E848
:100750008093BC008091BC0087FFFCCF8091BB00E0
:10076000089580910101811115C080E40E946C03FD
:100770008093010181110CC082E10E949603809355
:100780000101811105C08FEF0E9496038093010142
:100790000E948E0384B1807F84B985B1807F85B942
:1007A0008AB1837F8AB98BB1837F8BB93E98469893
:1007B00008950E946C05809301010E94B10380B3EB
:1007C0008C7080BB81B3836F81BBA5E3B1E0E3E4B0
:1007D000F1E08EE08E0F11921D928E13FCCF0C94DF
:1007E0005605BF92CF92DF92EF92FF920F931F9325
:1007F000CF93DF9380910101882379F080913401B8
:100800008F5F80933401811108C00E946C05809332
:100810000101811102C00E94FE0405E311E0C0E065
:10082000D0E0DD24D39482E0C82EEE24E394F12CB2
:10083000C730D10500F580910101811164C080E4C9
:100840000E946C0380930101811112C082E10E9419
:1008500096038093010181110BC0C7010C2E01C0CA
:10086000880F0A94EAF780950E949603809301010D
:100870000E948E0348C0CA30A1F028F4C83059F055
:10088000C93061F005C0CC3089F070F0CD3089F00E
:10089000209A289810C0219A29980DC0229A2A9847
:1008A0000AC0239A2B9807C0529A01C0539A5B98AA
:1008B00002C03E9A469890EA9A95F1F79FB17999CD
:1008C00002C082E001C080E091709D25982B7C9948
:1008D00002C084E001C080E0892B7D9902C038E02D
:1008E00001C030E0832B7E9902C020E101C020E0EE
:1008F000822B9FB19095991F9927991F9295990FD7
:10090000907E892B0FC080910101811149C080E444
:100910000E946C0380930101882379F1B12C0E941D
:100920008E038B2DF8019081981719F08083C09267
:1009300000010E94B10321960F5F1F4FCE30D105F9
:1009400009F076CF80910001882361F18150809376
:100950000001882339F08FE99FE00197F1F700C08B
:10096000000020C0A3E4B1E0E5E3F1E0CF01825F45
:1009700091919D938E13FCCF15C083E10E94960345
:10098000809301018111CACF81E40E946C0380939E
:1009900001018111C3CF0E94A703B82EB094BFCF2D
:1009A00080E0C0CF0E94FC0481E0DF91CF911F91D5
:1009B0000F91FF90EF90DF90CF90BF900895E82FB8
:1009C000F0E0ED5BFE4F8081089508950F931F9333
:1009D000CF93DF93C3E4D1E010E00C2F025F899145
:1009E00090E00E94931B180F0C13F9CF812FDF9119
:1009F000CF911F910F9108950C94CC0556985E9855
:100A000025982D9826982E9827982F988FEF90E06C
:100A1000909389008093880090938B0080938A0044
:100A200090938D0080938C00259A2D9A2FEF80E76C
:100A300092E0215080409040E1F700C00000269AEB
:100A40002E9A2FEF80E792E0215080409040E1F70E
:100A500000C00000279A2F9A2FEF80E792E02150E4
:100A600080409040E1F700C0000025982D982FEFBE
:100A700080E792E0215080409040E1F700C0000004
:100A800026982E982FEF80E792E0215080409040EA
:100A9000E1F700C0000027982F9856985E98259897
:100AA0002D9826982E9827982F98089589EA809354
:100AB000800089E08093810024982C983F988AB127
:100AC0008F748AB96E98479A8BB1806B8BB9769A7E
:100AD0000E94FE040C94CB0580E28093010180917A
:100AE000510181110EC00E94660381E08093510183
:100AF0002FEF83ED90E3215080409040E1F700C05C
:100B0000000080E40E946C038093010181112EC0DB
:100B10000E94960380930101811128C00E949603D0
:100B200080930101811122C08FE30E94960380937C
:100B3000010181111BC00E948E0380E40E946C039E
:100B400080930101811112C08CE00E949603809372
:100B5000010181110BC00E94960380930101811154
:100B600005C08FE30E949603809301010E948E03CB
:100B700080910101089561110BC0FC0182818823DD
:100B800021F085EE0E94A21103C085EE0E946A1238
:100B900080E090E0089508956091BD017091BE01DC
:100BA0008091BF019091C0010E949F1B56985E9852
:100BB00025982D9826982E9827982F98089581E0AB
:100BC000089581E008950C94E10508950F931F9313
:100BD000CF93DF938C01FC01C081D181CE010E94B3
:100BE000181ABE010E948F06EC01B8010E94E305AD
:100BF000882309F48DC0F8018281882309F44AC052
:100C000080915D0181111FC0C431F0E5DF0709F05B
:100C100051C00E94E50581E080935D010E94371C70
:100C200090935C0180935B011092540110925601E5
:100C300010925501109258011092570110925A01CA
:100C40001092590165C080915B0190915C010E94F6
:100C5000431C883C910570F480915401E82FF0E02A
:100C6000EE0FFF1FEB5AFE4FD183C0838F5F80933F
:100C700054014EC0C43880E5D80721F0C538D045AE
:100C800001F13AC0F8018281882341F010925201AB
:100C900082E01EC0C438E0E5DE0759F580915201BC
:100CA000811106C086E20E94A21186E20E946A12A9
:100CB00082E01CC0C438F0E5DF0741F3C538D045F9
:100CC000D9F4F8018281882331F01092530180E237
:100CD0000E94B9121DC080915301811106C087E2A4
:100CE0000E94A21187E20E946A1280E20E94C01252
:100CF0000FC0C538D04529F381E08093520180931D
:100D00005301C801DF91CF911F910F910C94DF0522
:100D100080E0DF91CF911F910F910895089596E0A3
:100D2000799FF001112494E5899FE00DF11D1124B4
:100D3000E60FF11DEE0FFF1FE65FFE4F85919491C8
:100D40000895880F991FFC01E657F0408591949112
:100D50000895880F991FFC01E65FFE4F85919491DD
:100D600008950F931F93CF93DF93EC01811520E338
:100D7000920750F5C11580E2D80708F0C3C0CB3BFD
:100D8000D10590F4C83AD10508F06AC0C53AD1053A
:100D900008F05BC0C430D10508F0D0C1219709F03C
:100DA000CAC101E010E00AC2CF3FD10511F008F03E
:100DB000C5C1C03FD10508F0A2C0CE01805E910937
:100DC000089708F4BBC1B7C1C13090E5D90709F451
:100DD000A2C020F5C0318FE4D80770F4C11590E4AB
:100DE000D90708F094C0C11521E3D20708F0A3C1C8
:100DF000DD278E01106CE2C1C115D04509F09BC101
:100E00000E941F158FEF94E32CE08150904020400A
:100E1000E1F700C000000E94921CD0C1C11597E507
:100E2000D90758F4C03121E5D20708F01CC1C431FC
:100E300080E5D80708F475C07EC1CE0190578115B2
:100E4000904108F078C1DF7073C1C53AD10509F44B
:100E500077C1C63AD10509F076C102E810E4AEC107
:100E6000C83AD10509F472C1C93AD10509F471C172
:100E7000CA3AD10509F470C1CB3AD10509F46FC162
:100E8000CC3AD10509F46EC1CD3AD10509F46DC152
:100E9000C03BD10509F46CC1CE3AD10509F46BC150
:100EA000CF3AD10509F46AC1C13BD10509F469C142
:100EB000C23BD10509F468C1C33BD10509F467C140
:100EC000C43BD10509F466C1C53BD10509F465C130
:100ED000C63BD10509F464C1C73BD10509F463C120
:100EE000C83BD10509F462C1C93BD10509F461C110
:100EF000CA3BD10509F460C100E014E45FC18E0172
:100F000010655CC1CE019F700E94A90658C1DF70B8
:100F10008E01106A53C18091DA0181608093DA01F9
:100F20004DC10E94371E811102C00E941D1E0E94E9
:100F3000541E90E09093FB018093FA01C23080E54B
:100F4000D80721F48091FA01816086C0C43090E511
:100F5000D90721F48091FA0182607EC0C63020E575
:100F6000D20721F48091FA01846076C0C83080E510
:100F7000D80719F48091FA0127C0CA3090E5D90743
:100F800021F48091FA01806167C0CC3020E5D2075E
:100F900021F48091FA0180625FC0CE3080E5D807ED
:100FA00021F48091FA01806457C0C03190E5D907DF
:100FB00021F48091FA0180684FC0C23120E5D20748
:100FC00029F48091FA018460886046C0C33080E5CE
:100FD000D80721F48091FA018E7F3EC0C53090E59C
:100FE000D90721F48091FA018D7F36C0C73020E502
:100FF000D20721F48091FA018B7F2EC0C93080E5A1
:10100000D80719F48091FA0126C0CB3090E5D907B2
:1010100021F48091FA018F7E1FC0CD3020E5D207E8
:1010200021F48091FA018F7D17C0CF3080E5D80779
:1010300021F48091FA018F7B0FC0C13190E5D9076F
:1010400021F48091FA018F7707C0C331D04531F484
:101050008091FA018B7F877F8093FA018091FA015A
:101060000E94581EABC08D2F99278F709927813011
:101070009105D9F49E012370332702C0880F991F70
:101080002A95E2F79C688E0144E0000F111F4A95F3
:10109000E1F700271370802B912B53E0CC0FDD1F5D
:1010A0005A95E1F7C076DD272FC08230910531F4E3
:1010B000DC2FCC278E01016F106A80C08330910530
:1010C00069F4CE018370992701E010E002C0000F9F
:1010D000111F8A95E2F7C8019C680FC08430910502
:1010E000B9F4CE018370992701E010E002C0000F2F
:1010F000111F8A95E2F7C8019A6823E0CC0FDD1F23
:101100002A95E1F7C07ED7708C010C2B1D2B56C0A1
:101110008530910531F4DC2FCC278E01046F106AE5
:101120004DC0069709F04AC0CF71DD27DC2FCC27D0
:101130008E01106243C000E010E040C08E013EC04E
:1011400001E810E43BC003E810E438C002EE14E408
:1011500035C009EE14E432C00AEE14E42FC005EBEA
:1011600014E42CC006EB14E429C007EB14E426C0F9
:101170000CEC14E423C00DEC14E420C003E815E4E7
:101180001DC00AE815E41AC002E915E417C004E915
:1011900015E414C001E216E411C003E216E40EC027
:1011A00004E216E40BC005E216E408C006E216E409
:1011B00005C007E216E402C00AE216E4C801DF91A6
:1011C000CF911F910F91089596E0799FF00111241E
:1011D00094E5899FE00DF11D1124E60FF11DEE0F3E
:1011E000FF1FE65FFE4F85919491803E9105E0F4EC
:1011F000803C910558F58133910509F46FC048F49E
:101200008932910509F463C08A32910509F46DC0F1
:1012100072C089339105E9F082389105D1F08533A8
:10122000910509F44DC067C0833E910581F138F402
:10123000803E9105B9F0823E9105D9F05CC0863EB2
:10124000910561F1873E9105A1F155C00E94A1066B
:1012500008952091FA0120FD02C021FF4CC080EECC
:1012600090E049C08091FA0180FFF9CF89E390E0D6
:1012700042C08091FA0182FF0EC08091FA0184FF82
:1012800003C080E090E037C083EE90E034C08091EE
:10129000FA0182FFF2CF82EE90E02DC08091FA0138
:1012A00083FF0BC08091FA0184FDEBCF87EE90E0C5
:1012B00022C08091FA0183FFF5CF86EE90E01BC03B
:1012C0008091FA0185FF07C089E290E014C0809107
:1012D000FA0185FFF9CF85E390E00DC08091FA0116
:1012E00086FF07C08AE290E006C08091FA0186FF7F
:1012F000F9CF81E390E00E94B106089508950C941F
:101300007E0980916E010895CF93DF9300D01F92E4
:10131000CDB7DEB79C018091F101843019F593E0DF
:1013200099833B832A839093E9008FEF9091E800A3
:10133000815095FD06C095ED9A95F1F70000811159
:10134000F5CF8091E80085FF0DC040E050E063E0FC
:1013500070E0CE0101960E94EE0B8091E8008E773E
:101360008093E8000F900F900F90DF91CF91089538
:10137000CF93DF9300D01F92CDB7DEB72091F1015C
:10138000243021F522E029839B838A8383E08093A4
:10139000E9008FEF9091E800815095FD06C095ED32
:1013A0009A95F1F700008111F5CF8091E80085FF53
:1013B0000DC040E050E063E070E0CE0101960E9475
:1013C000EE0B8091E8008E778093E8000F900F90ED
:1013D0000F90DF91CF9108952091F1012430F1F425
:1013E00022E02093E9002FEF3091E800215035FDF5
:1013F00006C035ED3A95F1F700002111F5CF2091A7
:10140000E80025FF0BC040E050E065E070E00E947E
:10141000EE0B8091E8008E778093E8000895CF93DB
:10142000DF93EC019091F101943009F046C0809176
:101430000C018823D9F080910D018823B9F0909395
:10144000E9008FEF9091E800815095FD06C095E18D
:101450009A95F1F700008111F5CF8091E80085FFA2
:101460002CC040E050E060E170E017C081E0809364
:10147000E9008FEF9091E800815095FD06C095ED51
:101480009A95F1F700008111F5CF8091E80085FF72
:1014900014C040E050E068E070E0CE010E94EE0B26
:1014A0008091E8008E778093E80080E1FE01AEE550
:1014B000B1E001900D928A95E1F7DF91CF91089507
:1014C0008091F001811109C00E94830D0E94E00DFE
:1014D0008091E20084608093E20008951092F00110
:1014E000089508950C94C7220E94281C0E94CD22C2
:1014F0000E9486100C947F0942E061EC81E00E941A
:10150000FD0C42E061EC82E00E94FD0C42E061ECE7
:1015100083E00E94FD0C42E161EC84E00C94FD0C40
:101520008091F301833009F455C030F4813071F0BB
:10153000823009F48EC008958A3009F47AC08B3065
:1015400009F460C0893009F09CC020C08091F2018C
:10155000813A09F096C08091E800877F8093E80087
:101560008091F6019091F701892B21F460E18EE5DD
:1015700091E003C060E080E090E070E00E94390CF0
:101580008091E8008B778093E80008958091F201C4
:10159000813209F076C08091F6019091F7010097B1
:1015A00019F0039709F06DC08091E800877F809360
:1015B000E8008091E80082FD05C08091F101811171
:1015C000F8CF5FC08091F10080936E018091E800B8
:1015D0008B7753C08091F201813A09F052C080911B
:1015E000F6019091F701892B09F04BC08091E8003A
:1015F000877F8093E8008091E80080FFFCCF809196
:101600000C0136C08091F2018132D9F58091F6014A
:101610009091F701892BA9F58091E800877F80934D
:10162000E8000E94320D8091F40180930C010C942B
:101630001F158091F201813221F58091E800877FAA
:101640008093E8000E94320D8091F50180936F0134
:1016500008958091F201813AA1F48091E800877F9A
:101660008093E8008091E80080FFFCCF80916F01BB
:101670008093F1008091E8008E778093E8000C94CD
:10168000320D089584B7877F84BF88E10FB6F89440
:1016900080936000109260000FBE90E080E80FB66B
:1016A000F89480936100909361000FBE0E94D51062
:1016B0000E94830D0E94E00D8091E200846080937F
:1016C000E20078940E9466100E94D71082E091E0B8
:1016D0000E9481100E94B5228091F101853069F449
:1016E0000E94EF1B8091EF018823B1F30E941A1C26
:1016F000882391F30E94D80BEFCF0E94DD10ECCF2E
:10170000292F332723303105C9F064F42130310506
:1017100081F02230310509F043C08DE690E026E8E3
:1017200034E042C021323105F1F02232310541F17D
:1017300037C082E190E023EF34E036C09927813052
:10174000910541F08230910541F0892B49F5E2E89D
:10175000F4E005C0EAE6F4E002C0E2E5F4E08491DA
:1017600090E09F0121C06430D8F4E62FF0E0EE0F46
:10177000FF1FEE5DFE4F2081318189E090E014C0B3
:10178000643070F470E0FB01EE0FFF1FE65EFE4F69
:1017900020813181FB01EA5EFE4F808190E004C030
:1017A00080E090E020E030E0FA013183208308956A
:1017B00080E189BD82E189BD09B400FEFDCF809141
:1017C000D8008F7D8093D8008091E0008260809364
:1017D000E0008091E00081FDFCCF0895CF92DF9280
:1017E000EF92FF920F931F93CF93DF93EC018B0146
:1017F0006A010E94510D811133C0C114D10439F026
:10180000F60180819181081B190BC80FD91FE12CAB
:10181000F12C0115110519F18091E80085FD16C024
:101820008091E8008E778093E800C114D10449F0DC
:10183000F60180819181E80EF91EF182E08285E057
:101840000FC00E94510D882321F30AC08991809313
:10185000F10001501109FFEFEF1AFF0ADACF80E023
:10186000DF91CF911F910F91FF90EF90DF90CF907C
:1018700008952091F8013091F9012617370748F0B3
:101880006115710539F42091E8002E772093E80066
:1018900001C0B90140E061157105A9F12091F10184
:1018A000222309F443C0253009F442C02091E80006
:1018B00023FD40C02091E80022FD32C02091E800C5
:1018C00020FFE9CF4091F3002091F20030E0342B6B
:1018D000FC01CF016115710559F02830310540F444
:1018E00081918093F100615071092F5F3F4FF1CFDB
:1018F00041E02830310509F040E02091E8002E77E2
:101900002093E800C8CF4111C9CF0AC08091F101EE
:10191000882361F0853061F08091E80083FD0AC082
:101920008091E80082FFF2CF80E0089582E0089580
:1019300083E0089581E008952091F8013091F90144
:101940002617370748F06115710539F42091E80032
:101950002E772093E80001C0B901FC0120E0611559
:10196000710591F18091F101882309F440C085301F
:1019700009F43FC08091E80083FD3DC08091E800FC
:1019800082FD2FC08091E80080FFE9CF2091F30015
:101990008091F20090E0922B6115710559F088302A
:1019A000910540F424912093F10031966150710922
:1019B0000196F2CF21E0089709F020E08091E8003D
:1019C0008E778093E800CBCF2111CCCF0AC08091D5
:1019D000F101882361F0853061F08091E80083FD9A
:1019E0000AC08091E80082FFF2CF80E0089582E093
:1019F000089583E0089581E00895982F973058F571
:101A00009093E900981739F07091EC002091ED0067
:101A10005091F00003C0242F762F50E021FF19C011
:101A20003091EB003E7F3093EB003091ED003D7F35
:101A30003093ED003091EB0031603093EB00709308
:101A4000EC002093ED005093F0002091EE0027FF72
:101A500007C09F5FD3CF8F708093E90081E0089526
:101A600080E008958091F20187FF11C08091E80025
:101A700082FD05C08091F1018111F8CF11C08091E4
:101A8000E8008B770BC08091F101882349F08091A9
:101A9000E80080FFF8CF8091E8008E778093E8001F
:101AA00008952091E4003091E50095E64091EC0026
:101AB000842F817040FF22C08091E80080FD1CC00F
:101AC0008091F101882391F0853091F08091EB00B5
:101AD00085FD10C04091E4005091E5004217530786
:101AE00029F39A01915011F784E0089582E0089556
:101AF00083E0089581E0089580E008954091E80032
:101B000042FFDECF08950E94F10D0E94F90DE0EE34
:101B1000F0E0808181608083E8EDF0E080818F7764
:101B2000808319BCA7EDB0E08C918E7F8C9380816F
:101B30008F7E80831092F00108950F931F93CF93AF
:101B4000DF930E94F10D0E94F90DC8EDD0E088816D
:101B50008F77888388818068888388818F7D888358
:101B600019BC1092F1011092ED011092EF01109248
:101B7000EE0100EE10E0F80180818B7F8083888188
:101B80008160888342E060E080E00E94FD0CE1EE2D
:101B9000F0E080818E7F8083E2EEF0E080818160E2
:101BA0008083808188608083F80180818E7F80833C
:101BB000888180618883DF91CF911F910F91089573
:101BC000E8EDF0E080818F7E8083E7EDF0E08081BA
:101BD0008160808384E082BF81E08093F0010C9477
:101BE0009D0DE8EDF0E080818E7F80831092E20011
:101BF00008951092DA001092E10008951F920F925A
:101C00000FB60F9211242F933F934F935F936F93CF
:101C10007F938F939F93AF93BF93EF93FF938091A5
:101C2000E10082FF0BC08091E20082FF07C080913B
:101C3000E1008B7F8093E1000E9465108091DA00C3
:101C400080FF1FC08091D80080FF1BC08091DA0008
:101C50008E7F8093DA008091D90080FF0DC080E1F3
:101C600089BD82E189BD09B400FEFDCF81E080938A
:101C7000F1010E94600A05C019BC1092F1010E9496
:101C80006E0A8091E10080FF19C08091E20080FF20
:101C900015C08091E2008E7F8093E2008091E20087
:101CA00080618093E2008091D80080628093D800A8
:101CB00019BC85E08093F1010E94720A8091E100D5
:101CC00084FF30C08091E20084FF2CC080E189BD98
:101CD00082E189BD09B400FEFDCF8091D8008F7DDF
:101CE0008093D8008091E1008F7E8093E100809105
:101CF000E2008F7E8093E2008091E2008160809319
:101D0000E2008091ED01882311F084E007C080910A
:101D1000E30087FD02C081E001C083E08093F10110
:101D20000E94740A8091E10083FF29C08091E20043
:101D300083FF25C08091E100877F8093E10082E0EE
:101D40008093F1011092ED018091E1008E7F8093EC
:101D5000E1008091E2008E7F8093E2008091E200BA
:101D600080618093E20042E060E080E00E94FD0C30
:101D70008091F00088608093F0000E94710AFF91CA
:101D8000EF91BF91AF919F918F917F916F915F91F3
:101D90004F913F912F910F900FBE0F901F9018956C
:101DA0001F920F920FB60F9211242F933F934F93D0
:101DB0005F936F937F938F939F93AF93BF93CF93D3
:101DC000DF93EF93FF93C091E900CF708091EC0017
:101DD000D82FD17080FDD0E81092E9008091F000FA
:101DE000877F8093F00078940E94140F1092E9008E
:101DF0008091F00088608093F000CD2BCF70C0936D
:101E0000E900FF91EF91DF91CF91BF91AF919F9149
:101E10008F917F916F915F914F913F912F910F9093
:101E20000FBE0F901F9018951F93CF93DF93CDB7E0
:101E3000DEB7AA970FB6F894DEBF0FBECDBFE2EFB4
:101E4000F1E088E08E0F9091F10091938E13FBCF1B
:101E50000E94900A8091E80083FF1FC18091F201E7
:101E60009091F301492F50E04A30510508F015C117
:101E7000FA01EA5AFF4F0C944F24803881F08238DF
:101E800009F00BC18091F6018F708093E900809179
:101E9000EB0085FB882780F91092E90006C080914D
:101EA000EE019091EF01911182609091E800977F8F
:101EB0009093E8008093F1001092F100C8C0282FA1
:101EC0002D7F09F0EAC0882319F0823061F0E5C067
:101ED0008091F401813009F0E0C0933009F080E096
:101EE0008093EF012BC08091F401811127C0809174
:101EF000F6018F7009F4D1C08093E9002091EB00C6
:101F000020FF1CC0933021F48091EB00806214C04C
:101F10009091EB0090619093EB0021E030E0A901FB
:101F200002C0440F551F8A95E2F74093EA001092D1
:101F3000EA008091EB0088608093EB001092E9004A
:101F40008091E800877F86C08111A7C01091F401BD
:101F50001F778091E3008078812B8093E30080914C
:101F6000E800877F8093E8000E94320D8091E800AE
:101F700080FFFCCF8091E30080688093E300111123
:101F800002C082E001C083E08093F10186C08058E6
:101F9000823008F082C08091F4019091F5018C3D6F
:101FA00053E0950779F583E08A838AE289834FB706
:101FB000F894DE01139620E03EE051E2E32FF0E0DA
:101FC00050935700E49120FF03C0E295EF703F5F0C
:101FD000EF708E2F90E0EA3010F0C79601C0C096E7
:101FE0008D939D932F5F243149F74FBF8091E80077
:101FF000877F8093E8006AE270E0CE0101960E943C
:10200000390C14C0AE014F5F5F4F6091F6010E9422
:10201000800BBC01009709F440C09091E800977FC5
:102020009093E80089819A810E949C0C8091E8003D
:102030008B778093E80031C0803879F58091E80093
:10204000877F8093E8008091ED018093F10080917B
:10205000E8008E778093E8000E94320D1EC0811147
:102060001CC09091F4019230C0F48091E800877F09
:102070008093E8009093ED010E94320D8091ED0174
:10208000811106C08091E30087FD02C081E001C09C
:1020900084E08093F1010E947C0A8091E80083FF34
:1020A0000AC08091E800877F8093E8008091EB0070
:1020B00080628093EB00AA960FB6F894DEBF0FBE45
:1020C000CDBFDF91CF911F9108950895CF93809157
:1020D000F1018823A1F0C091E900CF709091EC004C
:1020E000892F817090FD80E8C82B1092E9008091C3
:1020F000E80083FD0E94140FCF70C093E900CF91D8
:10210000089590937501809374010895E09174018E
:10211000F0917501309721F00190F081E02D099444
:1021200080E00895E0917401F0917501309721F0FD
:102130000280F381E02D09940895E0917401F091FB
:102140007501309721F00480F581E02D0994089500
:1021500020917201309173018217930771F090936F
:10216000730180937201E0917401F09175013097D1
:1021700021F00680F781E02D0994089520917001E7
:10218000309171018217930771F0909371018093E0
:102190007001E0917401F0917501309721F0008495
:1021A000F185E02D0994089508950C94D4100E94AF
:1021B0002E1C0E94D9030C94F01C9F92AF92BF92E8
:1021C000CF92DF92EF92FF920F931F93CF93DF9303
:1021D00000D000D000D0CDB7DEB70E94F1030DE0F3
:1021E00010E0AA24A394B12C902E802F0E94DF042B
:1021F000980129583E4F6901F901F080F826A1F4B1
:102200000150110988F78FEF89838A831B820E940E
:10221000371C8160782F9D838C8349815A816B8123
:102220008D810E9474112FC09091DA0191FF04C03A
:102230008E830E94E5048E8125E030E0A501022E08
:1022400001C0440F0A94EAF7E42E4F21C1F029831C
:102250009A828E2191E009F490E09B830E94371CC2
:102260008160782F9D838C8349815A816B818D8118
:102270000E947411F6018081E826E08204C021509A
:102280003109E0F6BDCF0E94D71F109176010E9460
:1022900086101817B9F00E94861080937601269652
:1022A0000FB6F894DEBF0FBECDBFDF91CF911F9167
:1022B0000F91FF90EF90DF90CF90BF90AF909F90E5
:1022C0000C947F0926960FB6F894DEBF0FBECDBFE3
:1022D000DF91CF911F910F91FF90EF90DF90CF9002
:1022E000BF90AF909F900895CF93DF93CDB7DEB7A7
:1022F0002B970FB6F894DEBF0FBECDBF4F83588724
:1023000069877A878B87DE01119686E0FD0111923D
:102310008A95E9F785E0FE01379601900D928A953E
:10232000E1F749815A816B817C818D819E810E9478
:10233000BD172B960FB6F894DEBF0FBECDBFDF9151
:10234000CF910895CF93882309F4C2C0C82F823853
:1023500059F40E94861081FDBBC089E30E94971A40
:102360000E94641B89E30CC0833879F40E948610B4
:1023700080FDAEC083E50E94971A0E94641B83E52E
:102380000E94D91ACF910C94641B843859F40E948E
:10239000861082FD9DC087E40E94971A0E94641BEC
:1023A00087E4EECF8CEF8C0F813A48F48C2F0E949B
:1023B0001A2281118DC08C2F0E94971AE3CF80E2E0
:1023C0008C0F883048F4C77081E001C0880FCA952F
:1023D000EAF70E941D1BD6CF8BE58C0F833078F473
:1023E000C53A29F0C63A31F083E890E005C081E8AB
:1023F00090E002C082E890E0CF910C94A81088E5AC
:102400008C0F833108F064C0C83A39F1C93A41F100
:10241000CA3A49F1CB3A51F1CC3A59F1CD3A61F18E
:10242000C03B69F1CE3A71F1CF3A79F1C13B81F10C
:10243000C23B89F1C33B91F1C43B99F1C53BA1F18A
:10244000C63BA9F1C73BB1F1C83BB9F1C93BC1F1EA
:10245000CA3BC9F180E090E038C082EE90E035C020
:1024600089EE90E032C08AEE90E02FC085EB90E0DC
:102470002CC086EB90E029C087EB90E026C08CEC66
:1024800090E023C08DEC90E020C083E891E01DC077
:102490008AE891E01AC082E991E017C084E991E0EE
:1024A00014C081E292E011C083E292E00EC084E2A7
:1024B00092E00BC085E292E008C086E292E005C09F
:1024C00087E292E002C08AE292E0CF910C94BE10C3
:1024D000CF910895882309F44BC0823859F40E94A3
:1024E000861081FF45C089E30E94971A0E94641BF1
:1024F00089E30CC0833871F40E94861080FF38C0D5
:1025000083E50E94971A0E94641B83E50E94D91AF2
:102510000C94641B843859F40E94861082FF28C0F2
:1025200087E40E94971A0E94641B87E4EFCF9CEF18
:10253000980F913A58F390E2980F983050F48770C2
:1025400091E001C0990F8A95EAF7892F0E94231B19
:10255000DFCF9BE5980F933020F480E090E00C945F
:10256000A810885A833120F480E090E00C94BE10CB
:102570000895882321F00E941D1B0C94641B08956C
:10258000882321F00E94231B0C94641B08957F92E2
:102590008F929F92AF92BF92CF92DF92EF92FF9273
:1025A0000F931F93CF93DF931F92CDB7DEB77C01BC
:1025B000C62E772EFC01058102950F701281111134
:1025C0000E943A1B0E94901A882379F0112369F027
:1025D00080E28C0D883048F082E00E94791A0E94D7
:1025E000901A91E0D82ED92601C0D12CE72DE29582
:1025F000EF70F0E0E05AFF4F0C944F24872D807F5E
:10260000072D0F70882311F00295007F112389F0A8
:10261000002309F490C180E28C0D883020F4802FD3
:102620000E941D1B03C0802F0E942D1B0E94641B53
:1026300082C18C2D0E946A12002309F495C180E2A8
:102640008C0D883020F4802F0E94231B03C0802F24
:102650000E94331B0E94641B87C1972D907F872D9A
:102660008F70903211F08295807FCC2021F0F1E0C4
:10267000CF16B1F01EC0112349F0002309F414C194
:10268000013009F011C10E944D1B6EC1002319F0E9
:10269000013009F469C189830E94501B89810AC1F4
:1026A000112321F0023008F05FC1FEC001115CC1AE
:1026B00001C1112321F0002309F4F6C03CC100231D
:1026C00009F4F8C03EC1872D86958695837090E009
:1026D000009719F0019761F047C1112321F08C2D6B
:1026E000972D937002C080E090E00E94A8103CC13A
:1026F000112321F08C2D972D937002C080E090E083
:102700000E94BE1031C18C2D112319F00E94DF1ED2
:1027100002C00E94471F0E94CC1F26C1872D8370D4
:1027200009F052C0111120C18C2D829586958770B9
:10273000880F880F9C2D9F70892E912CA12CB12C75
:10274000082E04C0880C991CAA1CBB1C0A94D2F742
:10275000C4FE14C00FE010E020E030E0B901A80191
:1027600004C0440F551F661F771F8A95D2F7CB010F
:10277000BA01609570958095909503C060E070E017
:10278000CB01272D26952695237030E02230310588
:1027900069F02330310589F0682979298A299B2934
:1027A0002130310571F00E940519DEC068297929B0
:1027B0008A299B290E942119D7C00E940519C501A9
:1027C000B4010E94E918D0C0112319F0872D81703F
:1027D00001C08695882309F4C7C08C2D8295869503
:1027E0008770880F880F9C2D9F70892E912CA12CAB
:1027F000B12C082E04C0880C991CAA1CBB1C0A947E
:10280000D2F7C4FE14C00FE010E020E030E0B901C0
:10281000A80104C0440F551F661F771F8A95D2F781
:10282000CB01BA01609570958095909503C060E0EA
:1028300070E0CB01272D269526952370422F50E07E
:102840004230510569F04330510589F068297929F2
:102850008A299B294130510571F00E94DF1984C0FB
:10286000682979298A299B290E94FB197DC00E9429
:10287000DF19C501B4010E94C31976C08C2D90E008
:10288000FC01E05EF109E531F10508F050C0E059C6
:10289000FF4F0C944F240C2D0F70872D8F71112337
:1028A00031F00E945C19802F0E94B9125DC00E9415
:1028B0007D19802F0E94C01257C0112339F00111D9
:1028C00053C0872D8F710E94A2194EC0023008F0AC
:1028D0004BC0F7CF112339F0872D8F710E945C19FF
:1028E00043C01123C9F3872D8F710E947D193CC00D
:1028F000112329F0872D8F710E94471935C00E943E
:102900003D1932C0112351F0172D1F71812F0E94E4
:102910005C1963E0812F0E94701A26C081E00E943A
:10292000791A023008F182E00E94791A1DC0112341
:1029300031F0002389F28C2D0E94A21115C00023D2
:1029400091F28C2D0E946A120FC0472D4F706C2D92
:10295000C7010E94BB050E94611806C0472D4F7039
:102960006C2DC7010E948E06DD20F9F00E946C1AC2
:1029700080FD1BC0F70112820E94661A0E945C193A
:10298000C7010E94E4140E94661A0F90DF91CF9154
:102990001F910F91FF90EF90DF90CF90BF90AF907D
:1029A0009F908F907F900C947D190F90DF91CF9125
:1029B0001F910F91FF90EF90DF90CF90BF90AF905D
:1029C0009F908F907F9008950F931F93CF93DF93E5
:1029D000EC01888199812B813C81232BB9F09F3FA9
:1029E00011F48F3F99F0CE010E94E605882371F023
:1029F000688179818A810E94621A8C010E94171A6B
:102A00000E94DE18B801CE010E94C712DF91CF915B
:102A10001F910F9108950E943A1B0E944A1B0E9429
:102A20000F1B0E94641B0E947D200E94CC1F80E02F
:102A300090E00E94A81080E090E00C94BE100E94EC
:102A40002A1B0C940B150E94571A292F22952F70C0
:102A500030E02C3031054CF42A3031056CF4225032
:102A6000310922303105A8F407C02C30310569F056
:102A70002F30310551F00DC0803F69F018F4803ED1
:102A800040F409C0843F29F406C093FB882780F9ED
:102A9000089580E0089581E00895CF93DF9300D0FA
:102AA00000D01F92CDB7DEB70F900F900F900F9010
:102AB0000F90DF91CF910895CF93DF9300D000D096
:102AC00000D0CDB7DEB726960FB6F894DEBF0FBEA6
:102AD000CDBFDF91CF9108951F93CF93DF93C09126
:102AE000850116E080918601C81799F0D0E01C9FFF
:102AF000F0011D9FF00D1124E957FE4F40815181D7
:102B000062817381848195810E945C152196C770D2
:102B1000E9CFDF91CF911F9108954091B701509176
:102B2000B8016091B9017091BA018091BB01909197
:102B3000BC010C945C158091BC0182958F7009F0EA
:102B400054C08091B901882309F44FC08091850158
:102B5000A09186016091B7017091B8014091BA01CE
:102B60005091BB01B6E08A1709F43FC090E04115CF
:102B70005105C1F17F3F11F46F3FA1F1B89FF00102
:102B8000B99FF00D1124E957FE4F218172132AC01D
:102B90002081621327C02281211124C02381348126
:102BA0002417350710F421503109241B350B283C1C
:102BB0003105C0F42091BC012F7020612093BC012D
:102BC00026E0289FF001299FF00D1124E457FE4FC5
:102BD00080818F708061808387EB91E00E94E41494
:102BE0000C946C1501968770BECF0895CF92DF923A
:102BF000EF92FF920F931F93CF93DF93CDB7DEB782
:102C000062970FB6F894DEBF0FBECDBF8C0185E092
:102C1000F801DE011D9601900D928A95E1F7D80129
:102C20004C9111965C91119712966C911297139694
:102C3000CD90DC9014973091B7017091B8018091DC
:102C4000BA019091BB01009709F46BC17F3F19F461
:102C50003F3F09F466C1E090B901EE2009F4C0C01D
:102C60002091BC01C816D90628F0F601E81BF90B23
:102C7000CF0104C0809590958C0D9D1DFF24F39489
:102C8000883C910578F0F12C207F09F0C6C07C2D9E
:102C9000D98AC88A89890E944D1587EB91E00E94E4
:102CA000E414B1C0822F807F09F046C0751314C0B0
:102CB000341312C0611110C02F7020612093BC0129
:102CC0000E948D1587EB91E00E94E4148091BC0175
:102CD000D80115968C932EC0CD2819F15F3F11F4C1
:102CE0004F3FF9F0F62E61111CC0809185012091B3
:102CF000860136E0821709F45AC090E0389FF0014F
:102D0000399FF00D1124E957FE4F7181571306C00A
:102D10007081471303C07281711103C001968770DF
:102D2000E9CFF62E662309F418C18091BC018160B9
:102D30008093BC01F12C11C1751308C0341306C077
:102D4000611104C08091BC01D801C3C04D875E876A
:102D50008D859E856A8B0E9423156A898823E1F1FF
:102D60006623D1F12091BC01822F82958F7090E073
:102D7000029774F08091B7019091B80198878F8382
:102D80001986DB86CA862C87CE0107960E94E4143A
:102D900086E0F801A7EBB1E001900D928A95E1F78A
:102DA0000E949B150E948D15FF24F394D6C04D8779
:102DB0005E878D859E850E94571A292F22952F7038
:102DC00030E0223031050CF0BCC09F7009F0B6C075
:102DD000805E883008F4C1C0C8010E94E414E4CFCA
:102DE000C816D90608F453C0F601E81BF90BCF0149
:102DF000883C910508F450C0F12C7C2DD98AC88AF2
:102E000089890E944D15E7EBF1E086E0DF011D9214
:102E10008A95E9F70E948D15A0C0751314C034136C
:102E200012C0611110C08091BC01F8018583C801F6
:102E30000E94E41486E0E7EBF1E0DF011D928A9541
:102E4000E9F7FE2C8AC04D875E878D859E856A8B4B
:102E50000E9423156A89882309F4BECF662309F4EA
:102E6000BBCF2091BC01822F82958F7090E002979A
:102E70000CF48ECF8091B7019091B8019A83898329
:102E80001B82DD82CC822E83CE0101967FCF80957E
:102E900090958C0D9D1DACCFF62E662309F49CCF2A
:102EA00075132EC034132CC02091BC0120FD1FC00F
:102EB000822F82958F70D9F0D80115962C93159793
:102EC0008F3049F08F5F982F9295907F822F8F706F
:102ED000892B15968C93C8010E94E41486E0F801B2
:102EE000A7EBB1E001900D928A95E1F793CF86E0D0
:102EF000F801A7EBB1E001900D928A95E1F72DC0A2
:102F00004D875E878D859E850E942315811140CF58
:102F10008091BC0181608093BC01C8010E94E414CF
:102F20001CC0662309F458CF4D875E878D859E852A
:102F30000E942315882309F44FCF2ACF811148CF4F
:102F40000CC0243031050CF047CF9F7009F440CFFE
:102F5000F8019581907F09F03BCF8F2D62960FB6D7
:102F6000F894DEBF0FBECDBFDF91CF911F910F91BF
:102F7000FF90EF90DF90CF9008951F93CF93DF9352
:102F8000CDB7DEB72C970FB6F894DEBF0FBECDBF1E
:102F90004F83588769877A878B879C87CE010796EE
:102FA0000E94F615882369F08F8198852A853B85D4
:102FB000232BF1F19F3F09F063C08F3F09F060C000
:102FC00037C086E0FE013796DE01119601900D9222
:102FD0008A95E1F76F817885EA85FB85309741F125
:102FE0007F3F11F46F3F21F12091860130E0C9014C
:102FF0000196877099274091850150E084179507C5
:1030000009F447C069837A83FD83EC8396E0929F3D
:10301000D001939FB00D1124A957BE4FFE013196E8
:1030200001900D929A95E1F7809386010E946C15AC
:1030300016E080918501909186018917C1F1189F52
:10304000C001112489579E4F0E94F615882379F1FB
:10305000E09185011E9FF0011124E957FE4F408148
:10306000518162817381848195810E945C15809178
:10307000850190E001968770992780938501D9CFCB
:103080004F81588569857A858B859C850E945C1562
:10309000CFCF0E941F151092860110928501E7EB99
:1030A000F1E086E0DF011D928A95E9F7C1CF2C9609
:1030B0000FB6F894DEBF0FBECDBFDF91CF911F9149
:1030C0000895EF92FF920F931F93CF93DF938C019C
:1030D000009709F46CC0F12CEE24E394E8012196EA
:1030E000F8018491843740F4843008F051C0813075
:1030F00081F0823019F15BC0853709F444C0A8F132
:103100009CE7980F903708F052C08F770E946A12A0
:1031100041C00E5F1F4FFE01C49180E28C0F8830CA
:1031200048F4C7708E2D01C0880FCA95EAF70E9437
:103130003D1B14C08C2F0E94A2112DC00E5F1F4F8B
:10314000FE01C49180E28C0F883058F4C7708E2D38
:1031500001C0880FCA95EAF70E94431B0E94641BB6
:103160001AC08C2F0E946A1216C00E5F1F4FFE01FC
:10317000C491CC2381F08FE99FE00197F1F700C063
:103180000000C150F6CF0E5F1F4FFE01F49003C048
:103190000E94A2118E018F2D882309F49FCFEFE9A1
:1031A000FFE03197F1F700C000008150F5CFDF91CB
:1031B000CF911F910F91FF90EF9008950895609324
:1031C000C1017093C2018093C3019093C4010C9418
:1031D0000B150F931F930091C1011091C201209113
:1031E000C3013091C401DC01CB01802B912BA22BB8
:1031F000B32B8093C1019093C201A093C301B093FC
:10320000C4011F910F910C940B150F931F93009104
:10321000C1011091C2012091C3013091C401DC01B0
:10322000CB0180239123A223B3238093C1019093E8
:10323000C201A093C301B093C4011F910F910C94DC
:103240000B150F931F930091C1011091C2012091A2
:10325000C3013091C401DC01CB0180279127A22753
:10326000B3278093C1019093C201A093C301B0938F
:10327000C4011F910F910C940B151092BD01109277
:10328000BE011092BF011092C0010C940B1541E0D9
:1032900050E060E070E004C0440F551F661F771FC8
:1032A0008A95D2F74093BD015093BE016093BF0150
:1032B0007093C0010C940B1541E050E060E070E0A9
:1032C00004C0440F551F661F771F8A95D2F780915F
:1032D000BD019091BE01A091BF01B091C001482BEA
:1032E000592B6A2B7B2B4093BD015093BE016093F9
:1032F000BF017093C0010C940B1541E050E060E0F9
:1033000070E004C0440F551F661F771F8A95D2F7DF
:1033100040955095609570958091BD019091BE014A
:10332000A091BF01B091C001482359236A237B2398
:103330004093BD015093BE016093BF017093C001E3
:103340000C940B1541E050E060E070E004C0440FC5
:10335000551F661F771F8A95D2F78091BD01909106
:10336000BE01A091BF01B091C001482759276A272B
:103370007B274093BD015093BE016093BF017093C2
:10338000C0010C940B150F931F930091BD01109178
:10339000BE012091BF013091C001DC01CB01802B27
:1033A000912BA22BB32B8093BD019093BE01A093D0
:1033B000BF01B093C0011F910F910C940B150F9397
:1033C0001F930091BD011091BE012091BF0130916A
:1033D000C001DC01CB0180239123A223B32380937E
:1033E000BD019093BE01A093BF01B093C0011F9196
:1033F0000F910C940B150F931F930091BD01109129
:10340000BE012091BF013091C001DC01CB018027BA
:103410009127A227B3278093BD019093BE01A0936B
:10342000BF01B093C0011F910F910C940B1508952B
:10343000CF92DF92EF92FF920F931F93CF93DF9380
:103440008C01C090C101D090C201E090C301F09006
:10345000C4018091BD019091BE01A091BF01B091C6
:10346000C001C82AD92AEA2AFB2ACFE1D0E0D70135
:10347000C6010C2E04C0B695A795979587950A941A
:10348000D2F780FF06C0B8018C2F0E94E408019794
:1034900021F4219760F780E001C08C2FDF91CF915C
:1034A0001F910F91FF90EF90DF90CF900895CF93F1
:1034B000DF93EC010E94181ABE010E94E408DF911C
:1034C000CF910895CB010E94571A08958091C501AC
:1034D00085958595859508958091C5018770089596
:1034E00098E0899F90011124262B2093C5010C940C
:1034F0005C192091C501809582238093C501982F86
:10350000977069F430E0482F552747FD50952417F0
:10351000350729F08595859585950C947D19089535
:103520009091C501977081E009F480E00895909131
:103530000C01992321F090910D01911109C0209166
:103540000E0130910F01F90132969FEF40E01FC04C
:10355000982F9695969596959F3050F5E0910E018F
:10356000F0910F01E90FF11D877021E030E0A90112
:1035700002C0440F551F8A95E2F7CA019181892B39
:10358000818308959F3F39F04F5F4E3041F0519154
:103590005813F8CF0DC05111F7CF942FF5CF9F3F9F
:1035A00039F0F901E90FF11D97FDFA95828308952D
:1035B000089590910C01992321F090910D019111A2
:1035C00009C020910E0130910F01F9013296205F60
:1035D0003F4F1FC0982F9695969596959F30F0F483
:1035E000E0910E01F0910F01E90FF11D877021E0CC
:1035F00030E0A90102C0440F551F8A95E2F7CA01C5
:10360000809591818923818308953196E217F3078C
:1036100029F090819813F9CF1082F7CF089581E0B7
:1036200090E0E0910E01F0910F01E80FF91F108278
:10363000019680319105A9F708959091D901892BC0
:103640008093D901089580959091D9018923809321
:10365000D90108951092D90108959091D801892B2C
:103660008093D801089580959091D8018923809303
:10367000D80108951092D80108959091D701892B0F
:103680008093D701089580959091D70189238093E5
:10369000D70108951092D70108958093C601089527
:1036A0001092C601089580910E0190910F01FC01C6
:1036B00031969C01205F3F4F80E0919191118F5F87
:1036C000E217F307D1F70895E0910E01F0910F0191
:1036D0008091D9018083E0910E01F0910F019081DA
:1036E0008091D801892B8083E0910E01F0910F0128
:1036F00090818091D701892B80838091C601882396
:1037000061F0E0910E01F0910F019081892B80838F
:103710000E94531B81111092C60180910E0190915D
:103720000F010C94921020E0009739F0AC01415049
:103730005109842395232F5FF7CF822F0895CF92CD
:10374000DF92EF92FF926C01EE24FF24C114D104AA
:10375000E104F10421F0C701B60120E101C020E03D
:10376000C72ED82EE92EFF24C114D104E104F104A0
:1037700019F0285FC701B6016B017C0154E0F69493
:10378000E794D794C7945A95D1F7C114D104E104B2
:10379000F10419F02C5FC701B6016B017C0142E016
:1037A000F694E794D794C7944A95D1F7C114D104FD
:1037B000E104F10419F02E5FC701B601DC01CB0171
:1037C000B695A79597958795892B8A2B8B2B09F012
:1037D0002F5F822FFF90EF90DF90CF900895809120
:1037E000F101843021F11092DB0120E488E190E0C6
:1037F0000FB6F894A895809360000FBE20936000E8
:1038000080E00E947F0983B7817F846083BF83B794
:10381000816083BF7894889583B78E7F83BF88E16A
:103820000FB6F89480936000109260000FBE089568
:10383000089508950E94181C0E94F1030E94191C0B
:103840000E94E60491E0811101C090E0892F089563
:103850000E941F150E9486100C947F0982E084BD8F
:1038600093E095BD9AEF97BD80936E0008952FB7B2
:10387000F8948091DC019091DD01A091DE01B0917E
:10388000DF012FBF0895CF92DF92EF92FF920F9347
:103890001F932FB7F8944091DC015091DD016091A6
:1038A000DE017091DF012FBF6A017B01EE24FF244E
:1038B0008C0120E030E0C016D106E206F30610F4D9
:1038C000415051099A01281B390BC9011F910F91D1
:1038D000FF90EF90DF90CF9008951F920F920FB658
:1038E0000F9211248F939F93AF93BF938091DC012C
:1038F0009091DD01A091DE01B091DF010196A11D43
:10390000B11D8093DC019093DD01A093DE01B093A3
:10391000DF01BF91AF919F918F910F900FBE0F90DC
:103920001F9018950E94830DF8942FEF87EA91E677
:10393000215080409040E1F700C0000087E090EB0C
:10394000DC018093FB019093FC01A093FD01B093F7
:10395000FE019CE088E10FB6F894A8958093600082
:103960000FBE90936000FFCFEF92FF920F931F93D3
:10397000CF93DF93D82FCDE08C2F0E94DF0405E09A
:1039800010E0E82EF12CC701002E02C09595879516
:103990000A94E2F780FF09C0602F7C2F80E00E942C
:1039A0008F06D81302C081E006C00150110958F7F4
:1039B000C15010F780E0DF91CF911F910F91FF90E0
:1039C000EF900895CF93C82F8CE20E94B41C8823F7
:1039D00021F08C2FCF910C94B41C80E0CF910895EE
:1039E000CF930E94371E811102C00E941D1EC5E6A2
:1039F000C15049F00E94F1038FE39CE90197F1F770
:103A000000C00000F5CF89E20E94E21C811113C1C1
:103A10008AE20E94E21C81110E941D1E85E00E9424
:103A2000E21C81110E94921C0E94421E8093DA01C6
:103A300087E00E94E21C8823A9F18BE10E94E21C2E
:103A4000882351F08091DA0181FB222720F991E04F
:103A5000922790FB81F90EC08EE00E94E21C882321
:103A600061F08091DA0182FB222720F991E0922710
:103A700090FB82F98093DA0115C080E10E94E21C7C
:103A80009091DA01882341F093FB222720F981E00D
:103A9000822780FB93F904C0892F809580FB90F9E1
:103AA0009093DA018091DA010E94461E0E94541E12
:103AB0008093FA0180EE0E94E21C882341F08091FD
:103AC000FA01982F909590FB80F98093FA0189E391
:103AD0000E94E21C882359F08091FA0181FB222781
:103AE00020F991E0922790FB81F98093FA0182EE10
:103AF0000E94E21C882359F08091FA0182FB222760
:103B000020F991E0922790FB82F98093FA0186EEEA
:103B10000E94E21C882359F08091FA0183FB22273E
:103B200020F991E0922790FB83F98093FA0183EECC
:103B30000E94E21C882359F08091FA0184FB22271D
:103B400020F991E0922790FB84F98093FA0185E3B4
:103B50000E94E21C882359F08091FA0185FB2227FC
:103B600020F991E0922790FB85F98093FA0181E397
:103B70000E94E21C882359F08091FA0186FB2227DB
:103B800020F991E0922790FB86F98093FA0181E178
:103B90000E94E21C882359F08091FA0187FB2227BA
:103BA00020F991E0922790FB87F98093FA018091A8
:103BB000FA010E94581E8091FA0187FB882780F93C
:103BC00080930D0187E20E94E21CC82F8EE10E94C3
:103BD000E21C8111C2608FE10E94E21C8111C4606D
:103BE00080E20E94E21C8111C86081E20E94E21C16
:103BF0008111C06182E20E94E21C8111C06283E2F5
:103C00000E94E21C8111C06484E20E94E21C8823AD
:103C100011F0C06802C0CC2329F08C2F0E944F1EE7
:103C20006C2F03C00E944B1E682F70E080E090E074
:103C3000CF910C94DF18CF9108956DEE7EEF80E068
:103C400090E00E94892460E082E090E00E94772466
:103C500060E083E090E00E94772460E084E090E000
:103C60000E94772460E085E090E00C94772480E067
:103C700090E00E94712421E08D3E9E4F09F020E0EB
:103C8000822F089582E090E00C946924682F82E0EE
:103C900090E00C94772483E090E00C946924682FE2
:103CA00083E090E00C94772484E090E00C94692405
:103CB000682F84E090E00C9477248091E20180FFEB
:103CC0000BC06091130185E0689FB00111247595C8
:103CD0006795759567952BC081FF09C060911301A9
:103CE00085E0689FB00111247595679520C082FF1B
:103CF00007C06091130185E0689FB001112417C0CF
:103D00009091E3019923D1F060911201961788F701
:103D10002091130185E0289F90011124929FA0011A
:103D2000939F500D112470E0CA010E943B2460381B
:103D3000710540F46115710539F002C065E070E06D
:103D4000862F08958FE7089581E008958091E2011C
:103D500080FF08C06091110170E0759567957595B9
:103D6000679521C081FF06C06091110170E07595D3
:103D7000679519C082FF04C06091110170E010C006
:103D80009091E3019923C1F0609110019617A0F77B
:103D900080911101899FC001112470E00E943B2491
:103DA0006038710528F46115710521F0862F08959A
:103DB0008FE7089581E0089561E070E0F4CF803FDF
:103DC00021F40E945D1E819504C0813F29F40E9468
:103DD0005D1E8093E6010895823F21F40E945D1EDE
:103DE000819504C0833F29F40E945D1E8093E50104
:103DF0000895893F19F40E94A61E05C08A3F31F438
:103E00000E94A61E81958093E70108958B3F21F4BF
:103E10000E94A61E819504C08C3F29F40E94A61E14
:103E20008093E8010895843F21F48091E40181604A
:103E300017C0853F21F48091E401826011C0863F64
:103E400021F48091E40184600BC0873F21F48091CC
:103E5000E401886005C0883F31F48091E40180610D
:103E60008093E40108958D3F21F48091E201816007
:103E70000BC08E3F21F48091E201826005C08F3F2C
:103E800029F48091E20184608093E2010895803FEB
:103E900039F48091E60187FF6CC01092E60169C099
:103EA000813F29F48091E6011816BCF362C090911D
:103EB000E501823F29F497FF5CC01092E50159C0EB
:103EC000833F19F41916CCF354C0893F41F4809113
:103ED000E70118160CF04DC01092E7014AC08A3F66
:103EE00029F48091E70187FF44C0F6CF8B3F39F476
:103EF0008091E80187FF3DC01092E8013AC08C3FF5
:103F000029F48091E8011816BCF333C0843F21F4F2
:103F10008091E4018E7F17C0853F21F48091E401F8
:103F20008D7F11C0863F21F48091E4018B7F0BC00F
:103F3000873F21F48091E401877F05C0883F31F4F9
:103F40008091E4018F7E8093E40113C08D3F21F4C2
:103F50008091E2018E7F0BC08E3F21F48091E201BF
:103F60008D7F05C08F3F29F48091E2018B7F809384
:103F7000E2018091E50181110EC08091E60181117D
:103F80000AC08091E701811106C08091E80181118A
:103F900002C01092E301089584EE91E00E949D100A
:103FA0000E94371C9093E1018093E00108951F93D4
:103FB000CF93DF938091E0019091E1010E94431C37
:103FC000AC019091E301992321F02091140130E09C
:103FD00006C0209115018AE0289F90011124421704
:103FE000530708F486C08091E501C091E601D091A5
:103FF000E7011091E801811107C0C11176C0D1110C
:1040000074C0111172C075C09F3F19F09F5F9093EB
:10401000E301181624F40E945D1E8093E50180914F
:10402000E50187FF05C00E945D1E81958093E50133
:104030001C1624F40E945D1E8093E6018091E60127
:1040400087FF05C00E945D1E81958093E601609107
:10405000E501662339F1C091E601CC2319F17727F8
:1040600067FD7095872F972F0E944C2323E333E33E
:1040700043E35FE30E94B0230E9419236093E501AC
:104080006C2F772767FD7095872F972F0E944C2301
:1040900023E333E343E35FE30E94B0230E94192349
:1040A0006093E6011D1624F40E94A61E8093E7018A
:1040B0008091E70187FF05C00E94A61E819580932D
:1040C000E701111624F40E94A61E8093E801809156
:1040D000E80187FF05C00E94A61E81958093E80134
:1040E000DF91CF911F910C94CC1F9F3F09F08ECF91
:1040F00096CFDF91CF911F910895E4EEF1E085E036
:10410000DF011D928A95E9F71092E3011092E20116
:104110000895833081F128F4813059F08230D1F054
:104120000895853009F449C0B8F1863009F456C0C5
:10413000089580911501262F30E0280F311D2F3F63
:10414000310524F4680F6093150108958FEF809373
:104150001501089580911401262F30E0280F311D9C
:104160002F3F310524F4680F6093140108958FEFF9
:1041700080931401089580911301262F30E0280FB9
:10418000311D2F3F310524F4680F6093130108950A
:104190008FEF80931301089580911201262F30E054
:1041A000280F311D2F3F310524F4680F6093120151
:1041B00008958FEF80931201089580911101262FA9
:1041C00030E0280F311D2F3F310524F4680F609334
:1041D000110108958FEF80931101089580911001CE
:1041E000262F30E0280F311D2F3F310524F4680FB2
:1041F0006093100108958FEF80931001089583302C
:1042000011F128F4813049F0823091F00895853021
:1042100081F120F18630C1F1089580911501681770
:1042200020F4861B809315010895109215010895BE
:1042300080911401681720F4861B8093140108955F
:1042400010921401089580911301681720F4861BC1
:104250008093130108951092130108958091120123
:10426000681720F4861B80931201089510921201A2
:10427000089580911101681720F4861B8093110125
:10428000089510921101089580911001681720F48B
:10429000861B8093100108951092100108950F93CA
:1042A0001F938D3109F46BC008F03FC08E3009F4C4
:1042B0007FC0C0F4873009F469C068F4863009F023
:1042C000B1C08091DA01817F8E7F8093DA0181E035
:1042D0008093EA01A8C0883009F4A2C08B3009F4A9
:1042E0009FC0A0C0863109F49BC078F4803109F4E6
:1042F00072C0813109F096C00E941F1590910D0186
:1043000081E0892780930D018BC0893109F488C031
:104310008B3109F087C08091DA0181FB222720F9D7
:1043200091E0922790FB81F94CC0853309F470C06D
:1043300048F4873209F46CC008F459C0893209F492
:1043400067C070C0833438F48A3308F04EC08833B5
:1043500009F466C067C0833409F45AC0883409F090
:1043600061C00E941F150FEF13ED20E301501040B4
:104370002040E1F700C000000E94921C51C00E9442
:10438000D3220E9486100E947F094AC09091DA01D0
:10439000892F8095817080FB90F929F09660986054
:1043A0009093DA0140C0997F977F9093DA0138C0EB
:1043B0008091DA0182FB222720F991E0922790FB7D
:1043C00082F98093DA01992359F18091DA018160B1
:1043D0008093DA0125C08091DA0183FB222720F93E
:1043E00091E0922790FB83F9ECCF895301C08D5166
:1043F00041E050E060E070E08A019B0104C0000FE2
:10440000111F221F331F8A95D2F7C901B80104C0BA
:1044100061E070E080E090E00E94DF180E941F15CC
:1044200081E001C080E01F910F91089580E0089520
:1044300080E00895CF93C82F8091EA01813079F010
:1044400018F08230E9F187C0E0910E01F0910F0180
:104450008081813169F0823209F07FC009C0E0912A
:104460000E01F0910F018081813111F0823261F4EF
:104470008C2F0E941622811104C08C2F0E944F2184
:104480001DC081E090E01AC08C2F0E94182281117B
:1044900014C0C43179F048F4CB3079F0C03109F060
:1044A00060C082E08093EA0108C0C93219F0C833C5
:1044B00021F057C01092EA0154C081E0817053C0CE
:1044C000C93289F118F5C43171F1A8F4C73009F087
:1044D00046C08AE08093150194E19093140193E023
:1044E000909313018093120188E08093110188E278
:1044F0008093100134C0CE51C63088F5EC2FF0E027
:10450000E65DFE4F80818093E90129C0CE34E9F059
:1045100020F4CB3421F56AE013C0C13579F0C235FF
:10452000F1F461E00DC08091E901882319F0109247
:10453000E90115C081E08093EA0115C061E006C081
:104540008091E9010E9489200AC06AE08091E90116
:104550000E94FF2004C01092EA0180E004C081E0C4
:1045600002C080E0ABCFCF910895E1E8F0E0808118
:10457000886080838081816080838FB7F89493E026
:104580009093890090ED909388008FBF0895EFE697
:10459000F0E08081826080830895EFE6F0E0808122
:1045A0008D7F80830895EFE6F0E0908182E0892797
:1045B000808308951F920F920FB60F9211242F93AC
:1045C0003F934F935F936F937F938F939F93AF939B
:1045D000BF93EF93FF938091EB019091EC010196D3
:1045E0009093EC018093EB01811103C082E00E9463
:1045F0007F09E091EC01E695E695F0E0E050FA4F96
:10460000E4918091EB018E1303C080E00E947F094A
:10461000FF91EF91BF91AF919F918F917F916F919A
:104620005F914F913F912F910F900FBE0F901F9070
:10463000189504D06894B1118DC0089570D088F099
:104640009F5790F0B92F9927B751A0F0D1F0660F7E
:10465000771F881F991F1AF0BA95C9F712C0B13099
:1046600081F077D0B1E0089574C0672F782F882744
:10467000B85F39F0B93FCCF3869577956795B395D8
:10468000D9F73EF490958095709561957F4F8F4F47
:104690009F4F0895E89409C097FB3EF4909580954C
:1046A000709561957F4F8F4F9F4F9923A9F0F92FF8
:1046B00096E9BB279395F695879577956795B79576
:1046C000F111F8CFFAF4BB0F11F460FF1BC06F5F5C
:1046D0007F4F8F4F9F4F16C0882311F096E911C06E
:1046E000772321F09EE8872F762F05C0662371F08F
:1046F00096E8862F70E060E02AF09A95660F771FA3
:10470000881FDAF7880F9695879597F9089557FDD2
:104710009058440F551F59F05F3F71F04795880F2F
:1047200097FB991F61F09F3F79F0879508951216C6
:1047300013061406551FF2CF4695F1DF08C0161672
:1047400017061806991FF1CF869571056105089423
:104750000895E894BB2766277727CB0197F908953A
:104760000BD078C069D028F06ED018F0952309F0EE
:104770005AC05FC01124EECFCADFA0F3959FD1F3DA
:10478000950F50E0551F629FF001729FBB27F00DFF
:10479000B11D639FAA27F00DB11DAA1F649F662754
:1047A000B00DA11D661F829F2227B00DA11D621FA3
:1047B000739FB00DA11D621F839FA00D611D221F5D
:1047C000749F3327A00D611D231F849F600D211D41
:1047D000822F762F6A2F11249F5750408AF0E1F0E4
:1047E00088234AF0EE0FFF1FBB1F661F771F881F2D
:1047F00091505040A9F79E3F510570F014C0AACFC8
:104800005F3FECF3983EDCF3869577956795B79517
:10481000F795E7959F5FC1F7FE2B880F911D969541
:10482000879597F9089597F99F6780E870E060E0B1
:1048300008959FEF80EC089500240A941616170639
:1048400018060906089500240A9412161306140681
:1048500005060895092E0394000C11F4882352F0E4
:10486000BB0F40F4BF2B11F460FF04C06F5F7F4F9C
:104870008F4F9F4F089597FB072E16F4009407D093
:1048800077FD09D00E94552407FC05D03EF4909591
:1048900081959F4F0895709561957F4F0895EE0F14
:1048A000FF1F0590F491E02D0994AA1BBB1B51E159
:1048B00007C0AA1FBB1FA617B70710F0A61BB70B90
:1048C000881F991F5A95A9F780959095BC01CD0135
:1048D0000895F999FECF92BD81BDF89A992780B5C8
:1048E0000895A8E1B0E042E050E00C949124262F16
:1048F000F999FECF92BD81BDF89A019700B40216D6
:1049000039F01FBA20BD0FB6F894FA9AF99A0FBE83
:1049100008950196272F0E9478240C947724DC01B7
:10492000CB01FC01F999FECF06C0F2BDE1BDF89ABA
:10493000319600B40D9241505040B8F70895F89464
:02494000FFCFA7
:10494200022081090F0AEC09B80984090101C70193
:1049520028080A03140A3F4D3639C10574053E057D
:1049620005059804B104CA04E30401020304050620
:044972000708090029
:00000001FF
